:020000040800F2
:100000000000022089390008813400088334000888
:100010008534000887340008893400080000000097
:100020000000000000000000000000008B34000809
:100030008D340008000000008F340008913400085F
:10004000D9390008D9390008D9390008D939000848
:10005000D9390008D9390008D9390008D939000838
:10006000D9390008D9390008D9390008D939000828
:10007000D9390008D9390008D9390008D939000818
:10008000D9390008D9390008D9390008D939000808
:10009000D9390008D9390008D9390008D9390008F8
:1000A000D9390008D9390008D9390008D9390008E8
:1000B000D9390008D9390008D9390008D9390008D8
:1000C000D9390008D9390008D9390008D9390008C8
:1000D000D9390008D9390008D9390008D9390008B8
:1000E000D9390008D9390008D9390008D9390008A8
:1000F000D9390008D9390008D9390008D939000898
:10010000D9390008D9390008D9390008D939000887
:1001100095340008D9390008D9390008D9390008C0
:10012000D9390008D9390008D9390008D939000867
:10013000D9390008D9390008D9390008D939000857
:10014000D9390008D9390008D9390008A134000884
:10015000D9390008D9390008D9390008D939000837
:10016000D9390008D9390008D9390008D939000827
:10017000D9390008D9390008D93900080000000031
:08018000D9390008D939000843
:1001880010B5054C237833B9044B13B10448AFF3C9
:1001980000800123237010BDC8010020000000006A
:1001A800183C000808B5034B1BB103490348AFF3DB
:1001B800008008BD00000000CC010020183C0008A9
:1001C80053B94AB9002908BF00281CBF4FF0FF31B6
:1001D8004FF0FF3000F07AB9ADF1080C6DE904CEAC
:1001E80000F006F8DDF804E0DDE9022304B070470A
:1001F8002DE9F0478C460D460446089E002B51D148
:100208008A4217466DD9B2FA82FEBEF1000F0BD0B2
:10021800CEF1200C01FA0EF520FA0CFC02FA0EF7CA
:100228004CEA050C00FA0EF44FEA174A250CBCFB01
:10023800FAF81FFA87F90AFB18CC45EA0C4508FBBF
:1002480009F3AB420AD9ED1908F1FF3280F0238196
:10025800AB4240F22081A8F102083D44ED1AA4B255
:10026800B5FBFAF00AFB105544EA054400FB09F90E
:10027800A14509D9E41900F1FF3380F00A81A145AD
:1002880040F2078102383C44A4EB090440EA0840E4
:100298000021002E61D024FA0EF40023346073602C
:1002A800BDE8F0878B4207D9002E54D0002186E89C
:1002B80021000846BDE8F087B3FA83F1002940F031
:1002C8008E80AB4202D3824200F2FA80841A65EB38
:1002D80003050120AC46002E3FD086E81010BDE88B
:1002E800F08712B90127B7FBF2F7B7FA87FEBEF11C
:1002F800000F34D1EB1B3A0C1FFA87FC0121B3FB2A
:10030800F2F8250C02FB183345EA03450CFB08F309
:10031800AB4207D9ED1908F1FF3002D2AB4200F227
:10032800D1808046ED1AA3B2B5FBF2F002FB10555E
:1003380043EA05440CFB00FCA44507D9E41900F185
:10034800FF3302D2A44500F2B8801846A4EB0C048F
:1003580040EA08409DE731463046BDE8F087CEF1D7
:10036800200405FA0EF307FA0EF720FA04F83A0CFF
:1003780025FA04F448EA0308B4FBF2F14FEA1845F9
:1003880002FB11441FFA87FC45EA044501FB0CF304
:10039800AB4200FA0EF409D9ED1901F1FF3080F0F3
:1003A8008A80AB4240F2878002393D44EB1A1FFA3B
:1003B80088F5B3FBF2F002FB103345EA034500FB76
:1003C8000CF3AB4207D9ED1900F1FF386FD2AB42FD
:1003D8006DD902383D44EB1A40EA01418FE7C1F17B
:1003E800200722FA07F88B4005FA01F448EA0303CC
:1003F80020FA07FE4FEA134CFD404EEA040EB5FB07
:10040800FCF94FEA1E440CFB19551FFA83F844EA1D
:10041800054509FB08F4AC4202FA01F200FA01FAB8
:1004280008D9ED1809F1FF3043D2AC4241D9A9F1FE
:1004380002091D442D1B1FFA8EFEB5FBFCF00CFBB8
:1004480010554EEA054400FB08F8A04507D9E41802
:1004580000F1FF3529D2A04527D902381C4440EACB
:100468000940A4EB0804A0FB02894C45C6464D464A
:1004780015D312D056B1BAEB0E0364EB050404FA97
:1004880007F7CB401F43CC40376074600021BDE8BC
:10049800F0871846F8E69046E0E6C245EAD2B8EB9F
:1004A800020E69EB03050138E4E72846D7E7404622
:1004B80091E78146BEE7014678E702383C4445E7C4
:1004C800084608E7A8F102083D442BE7704700BF3B
:1004D80038B50E4A0E4B054618784FF47A73B3FBBD
:1004E800F0F31068B0FBF3F000F0A8F8044658B930
:1004F8000F2D09D8024629464FF0FF3000F05EF86C
:10050800044B20461D6038BD012038BD1C01002069
:10051800000000200400002008B50B4B1A6842F4C4
:1005280000721A601A6842F480621A601A6842F40B
:1005380080721A60032000F02FF80020FFF7C8FF30
:1005480002F03EFF002008BD003C0240034A044B75
:1005580011681B780B441360704700BFF801002036
:1005680000000020014B1868704700BFF801002008
:1005780038B50446FFF7F6FF631C1CBF054B1B7814
:10058800054618BFE418FFF7EDFF401B8442FAD870
:1005980038BD00BF00000020074AD36823F4E06399
:1005A8001B041B0C43F0BF63000243F4003300F448
:1005B800E0600343D360704700ED00E0174B30B5AF
:1005C800DC68C4F30224C4F10703251D042B28BFEB
:1005D8000423062D4FF0010505FA03F303F1FF3359
:1005E8008CBF033C00241940A14005FA04F4013CE7
:1005F8002240002842EA01024FEA0212AFBF00F18E
:10060800604000F00F00064BD2B2A5BF00F5614074
:10061800D2B21A5480F8002330BD00BF00ED00E0CC
:1006280014ED00E04209012300F01F0003FA00F076
:10063800014B43F82200704700E100E00138B0F1B7
:10064800807F0AD2064B074A5860F02182F82310AF
:100658000020072298601A6070470120704700BF89
:1006680010E000E000ED00E090F83530022B03D0F8
:1006780080234365012070470268052380F83530E0
:10068800136823F001031360002070472DE9F04F31
:1006980085B00B68DFF8AC81684ADFF8AC9101934C
:1006A80000234FF0010E019C0EFA03FE0EEA040629
:1006B800B64540F0AE804C6824F01007022F16D1E2
:1006C8004FEAD30A00EB8A0A03F0070BDAF8205046
:1006D8004FEA8B0B4FF00F0C0CFA0BFC25EA0C0CB5
:1006E8000D6905FA0BF545EA0C05CAF820504FEAE2
:1006F800430A0325D0F800B005FA0AF5ED4304F0E3
:10070800030C0BEA050B0CFA0AFC013F4CEA0B0C34
:10071800012FC0F800C011D8876807EA050BCF6819
:1007280007FA0AFC4CEA0B078760476827EA0E0EAF
:10073800C4F300179F4047EA0E074760C7683D406B
:100748008F6807FA0AF73D43C560E50061D54FF0A9
:10075800000BCDF80CB0D8F84470394D47F48047F9
:10076800C8F84470D8F8447007F480470397039F8B
:1007780023F0030707F1804707F59C3703F0030CC4
:10078800D7F808A04FEA8C0C4FF00F0E0EFA0CFEAB
:10079800A8422AEA0E0E43D005F58065A84241D04A
:1007A80005F58065A8423FD005F58065A8423DD093
:1007B80005F58065A8423BD048453BD005F5006566
:1007C800A84239D005F58065A84214BF0825072539
:1007D80005FA0CF545EA0E05BD601568F74314F4F3
:1007E800803F0CBF3D4035431560556814F4003F09
:1007F8000CBF3D4035435560956814F4801F0CBF0D
:100808003D4035439560D568A40254BF3D4035430B
:10081800D5600133102B7FF444AF05B0BDE8F08FED
:100828005D46D5E70125D3E70225D1E70325CFE7C4
:100838000425CDE70525CBE70625C9E7003C01409F
:100848000000024000380240001402400AB18161F1
:1008580070470904FBE7F0B506468BB0002864D062
:100868000323344680F8B93302F0F2FE54F8100B33
:1008780001F0D6F90FCC6D460FC50FCC0FC594E823
:10088800030085E80300371D97E80E00306801F083
:1008980087F90021306801F0C9F900213346324652
:1008A80006F110040125084682F83810D187013175
:1008B8000F2982F8395082F83B0010645064D064E4
:1008C80002F11C02F0D10022D6F800E0114602F134
:1008D800400083F8F821DA870EEB800001320F2AF6
:1008E80083F8F91183F8FB11C3F80012C3F8041256
:1008F800C3F80C12416003F11C03E8D10FCC6D461C
:100908000FC50FCC0FC594E8030085E803007046B7
:1009180097E80E0001F0A2F9012386F8B933306890
:1009280001F0BFFC00200BB0F0BD0120FBE790F800
:10093800B833012B10B504460CD0012380F8B83326
:10094800006801F0A2FC206801F064F9002084F836
:10095800B80310BD022010BD2DE9F04FD0F800906B
:1009680087B00446484601F0D6FC0290002840F0C3
:100978002E81206801F0A1FC002800F02881206861
:1009880001F09BFC850748BF2268206842BF536975
:1009980003F00203536101F090FC10F400250AD023
:1009A800206801F08EFC09F530660746A24600254E
:1009B800002F40F00F81206801F07FFC41030BD528
:1009C800206801F086FC2646039009F5106800258A
:1009D800039B002B40F03F81206801F06EFC00284B
:1009E8000DDAD9F8043823F00103C9F80438204691
:1009F80002F0A4FE2268536903F0004353612068A3
:100A080001F05BFC06050BD5D9F80838D80702D5E4
:100A1800204602F07BFE2268536903F400635361A9
:100A2800206801F04AFCC10437D509F500667368EF
:100A3800206823F001037360102101F0ABF96168AD
:100A480009F51063FF220298884240F092814FF026
:100A5800FF33B361F36943F00113F361236B002B98
:100A680000F08F81D6F8843043F00B03C6F8843049
:100A7800736C43F00B037364D9F80038217C206849
:100A880023F4FE63C9F8003804F56F7201F062FCC4
:100A98002268536903F480535361206801F00DFC08
:100AA80082041DD5206801F03AFC2068C36823F44D
:100AB8007053C36001F097F9002840F06B812268F9
:100AC800E0604FF400736361D36843F41053D3605C
:100AD800204602F00AFE2268536903F4005353616A
:100AE800206801F0EAFBC3062BD52268936923F03E
:100AF80010039361D9F82060C6F34343022B06F034
:100B08000F0840F0A88147F6F0731E4214D01C2746
:100B180007FB0847C6F30A163246D7F804124846B8
:100B280001F05DFBD7F804323344C7F80432D7F834
:100B380010321E44C7F810622268936943F010030C
:100B48009361206801F0B9FB070707D5204602F03A
:100B5800C8FD2268536903F008035361206801F057
:100B6800ACFBC60208D5E9B2204602F0EFFD2268C8
:100B7800536903F480135361206801F09EFB8002DF
:100B880008D5E9B2204602F0DDFD2268536903F476
:100B980000135361206801F090FB410007D52046FF
:100BA80002F0D8FD2268536903F08043536120683E
:100BB80001F083FB42070AD523685D686B0702D5FD
:100BC800204602F0CBFD23685A6815435D6007B0E4
:100BD800BDE8F08FF80738D55FFA85FB59462068DD
:100BE80001F07FFB10F0010F804621D0216901231D
:100BF8009942B3600CD13169DAF80002C1F31201ED
:100C0800411ACAF81012DAF804120844CAF80402A1
:100C18005946204602F054FD2169012908D13DB901
:100C2800D4F80C2222B904F56F72206801F092FB07
:100C380018F0080F04D0204602F03CFD0823B360EA
:100C480018F0100F1CBF1023B36001357F08203641
:100C58000AF11C0AACE6039BDA0758D55FFA85FB54
:100C68005946206801F047FBC307074620D5D9F845
:100C780034380121A94023EA0103C9F83438012393
:100C8800C8F808302369012B01BF736C326C9B18BC
:100C980073645946204602F01CFD2169012907D1D9
:100CA80035B9E36C23B904F56F72206801F052FB83
:100CB800380744BF0823C8F80830F90644BF102392
:100CC800C8F808307A0644BF4023C8F80830BB0784
:100CD80044BF0223C8F808303F0618D52368049398
:100CE800F76C336DFF1A336C9F4228BF1F46049B75
:100CF80003F5106307F1030A03EB45134FEA9A0A59
:100D08000593059B9B699BB2534508D82FB3039B5A
:100D18005B08013503931C3608F1200858E6326D4C
:100D2800F36C9342F2D9002BF0D0376C04989B1ADD
:100D38009F4228BF1F46237C00935A46BBB2716C62
:100D480001F039FA736C3B447364336D07F1030A9D
:100D58003B444FEA9A0A3365D3E7049B012203F523
:100D6800006BD3F83438AA4023EA0203CBF83430B6
:100D7800CDE702989A600130C3F808220290203328
:100D880061E6736943F00B037361336943F00B0346
:100D9800336171E60323E3604023636100F0F8FBED
:100DA800344B354A03449342236804D8DA6842F442
:100DB8007052DA608CE6314A314902448A4203D8DB
:100DC800DA6842F46052F4E7A0F574022D49A2F5FE
:100DD80010528A4203D8DA6842F45052E9E7A0F187
:100DE80083722949A2F5E7428A4203D8DA6842F4B5
:100DF8004052DEE7254A264902448A4203D8DA6887
:100E080042F43052D5E7234A234902448A4203D8A0
:100E1800DA6842F42052CCE7204A214902448A4247
:100E280003D8DA6842F41052C3E7A0F1B7721D493B
:100E3800A2F558528A4203D8DA6842F40052B8E759
:100E4800194A1A4902448A42DA6894BF42F4E052C5
:100E580042F4C052ADE7062B7FF46EAE082204F5CB
:100E68006F7148461C2701F0BAF907FB0847C6F31B
:100E78000A165CE6405327FFFF340C00401E1BFF98
:100E88003F420F007F4F12001FD6130060B6E5FEE9
:100E98005FE3160000D3CEFE3F771B00C05BB3FEB6
:100EA800BF9121001F753800E05459FEDF9C4100B6
:100EB80090F8B833012B10B5044609D0012380F807
:100EC800B833006801F0D1F9002084F8B80310BDE8
:100ED800022010BD70B54EB2002E04464FF01C051E
:100EE80001F07F00B5BF05FB004105FB014138312A
:100EF80001F5FC71C0B2002EB8BFC880022BCB70C0
:100F08004FEAD67504BF00230B7108704D7094F832
:100F1800B8338A60012B09D0012384F8B8332068DC
:100F280000F07CFF002084F8B80370BD022070BD7B
:100F38004BB2002B10B54FF01C02044601F07F00A5
:100F4800B5BF02FB004102FB0141383101F5FC71DC
:100F5800DB0F08704B7094F8B833012B09D00123CC
:100F680084F8B833206800F098FF002084F8B803AC
:100F780010BD022010BD38B501F07F051C2404FB0C
:100F8800050104FB050401F5FC71C4F80C320023CB
:100F9800C4F80422C4F8103284F8F93184F8F851FE
:100FA80003690068012B08BFC4F80822DAB21DB92A
:100FB80001F094F8002038BD00F0CAFFFAE71C23BE
:100FC80001F00F0103FB0101B1F81002704738B5B9
:100FD80001F07F051C2404FB050104FB05043831DE
:100FE800E364002323650123626484F8393084F8BC
:100FF800385003690068012B08BFA264DAB21DB932
:1010080001F06CF8002038BD00F0A2FFFAE738B50F
:101018004BB2002B01F07F054FF01C02B5BF02FB5D
:10102800050102FB0101383101F5FC710122DB0FDA
:10103800EDB28A700D704B7090F8B8339342044645
:101048000FD080F8B823006801F0D7F82DB904F55F
:101058006F72217C206801F07DF9002084F8B803C4
:1010680038BD022038BD38B54BB2002B05464FF0CD
:101078001C0201F07F00B5BF02FB005102FB0151C9
:10108800383101F5FC71DB0F00248C7008704B704F
:1010980095F8B833012B09D0012385F8B8332868AF
:1010A80001F0CAF885F8B843204638BD022038BD9B
:1010B800006870B5436A21B943EA0243836200209D
:1010C80070BD846A002503EB14434E1EECB2B44293
:1010D80005F1010506DB3F3100EB810043EA0243DD
:1010E8004360ECE7403400EB8404646803EB14438A
:1010F800ECE7036800205962704700002DE9F341CE
:10110800044618B9012002B0BDE8F0810368DD0784
:1011180010D42368980758D423681A0700F19A80D6
:1011280023685B0700F1B880A269002A40F01981A2
:101138000020E8E7A64B9A6802F00C02042A07D0C0
:101148009A6802F00C02082A0AD15B68590207D58E
:101158009F4B1B689A03DCD56368002BD9D1D1E774
:1011680063689B4DB3F5803F11D12B6843F48033FE
:101178002B60FFF7F7F9964D06462B689B03C8D4FA
:10118800FFF7F0F9801B6428F7D90320BBE7B3F514
:10119800A02F04D12B6843F480232B60E5E72A684D
:1011A80022F480322A602A6822F480222A60002BE6
:1011B800DFD1FFF7D7F906462B689F03A9D5FFF7BC
:1011C800D1F9801B6428F7D9DFE7814B9A6812F0C0
:1011D8000C0F07D09A6802F00C02082A11D15B683C
:1011E8005E020ED47A4B1A68950702D5E268012A86
:1011F80088D11A68216922F0F80242EAC1021A600D
:101208008AE7E268734BB2B101221A60FFF7AAF9C4
:101218006F4D06462B68980707D52B68226923F07F
:10122800F80343EAC2032B6076E7FFF79BF9801BBC
:101238000228EFD9A9E71A60FFF794F9644D06462A
:101248002B6899077FF568AFFFF78CF9801B022898
:10125800F6D99AE76269604B7AB101221A60FFF702
:1012680081F95B4D06466B6F9F073FF559AFFFF756
:1012780079F9801B0228F6D987E71A60FFF772F917
:10128800534D06466B6F98077FF54AAFFFF76AF92B
:10129800801B0228F6D978E74D4B1A6C12F0805261
:1012A80028D101921A6C42F080521A641B6C03F028
:1012B80080530193019B0126484D2B68D9051BD506
:1012C800A368434D012B27D12B6F43F001032B67F4
:1012D800FFF748F93E4D074641F288382B6F9B07C8
:1012E80039D5002E3FF420AF394A136C23F08053D0
:1012F800136419E70026DFE72B6843F480732B603B
:10130800FFF730F907462B68DA05D9D4FFF72AF931
:10131800C01B0228F7D938E7052B04D12B6F43F0FF
:1013280004032B67D0E72A6F22F001022A672A6F8D
:1013380022F004022A67002BCAD1FFF713F941F201
:10134800883807462B6F9807CBD5FFF70BF9C01BDA
:101358004045F7D919E7FFF705F9C01B4045BDD946
:1013680013E71B4DAB6803F00C03082B3FF4CAAE20
:101378001B4E0023022A336034D1FFF7F3F80746E7
:101388002B6899011ED4226AE3691343626A43EA0F
:101398008213E26A43EA0263A26A0D4C5208013AD8
:1013A80043EA02436B6001233360FFF7DBF805462D
:1013B80023689A013FF5BCAEFFF7D4F8401B02281A
:1013C800F6D9E2E6FFF7CEF8C01B0228D8D9DCE64A
:1013D8000038024000004742800E4742007000403B
:1013E80060004742FFF7BEF804462B689B017FF573
:1013F8009FAEFFF7B7F8001B0228F6D9C5E600BF75
:10140800134908B58B6803F00C03042B03D0082B91
:1014180003D0104808BD104808BD4A684B684968A1
:1014280013F4800314BF0C480A48C1F3881118BF8D
:10143800002302F03F02A1FB0001FEF7C1FE044BAE
:101448005B68C3F3014301335B00B0FBF3F008BDF5
:10145800003802400024F40000127A002DE9F0411F
:101468000D46044610B90120BDE8F081444B1A68C6
:1014780002F00F028A4228D321688F072DD4C807AB
:1014880040D43F4B1A6802F00F02954266D3226897
:1014980051076CD4130707D53A4A2169936823F496
:1014A800604343EAC1039360FFF7AAFF354B364A0E
:1014B8009B68C3F30313D35CD840344B18600020F7
:1014C800FFF706F80020BDE8F081CAB21A701B6861
:1014D80003F00F039942C6D1CEE72A4B11F0040F4F
:1014E8001EBF9A6842F4E0529A600E0742BF9A689B
:1014F80042F460429A609A68A06822F0F0020243BF
:101508009A60BCE762681F4B012A1DD11B6813F45F
:10151800003FA8D01B4EB36823F003031343B36006
:10152800FFF720F841F288380746B368626803F08D
:101538000C03B3EB820FA4D0FFF714F8C01B40458F
:10154800F3D90320BDE8F081911E01291B6802D858
:1015580013F0007FDDE713F0020FDAE7EAB21A7042
:101568001B6803F00F039D427FF47DAF8FE70549A9
:10157800E0688B6823F4E05303438B608AE700BF7D
:10158800003C024000380240303C00081C010020AA
:10159800014B1868704700BF1C010020044B054A26
:1015A8009B68C3F38223D35C034A1068D840704712
:1015B80000380240403C00081C010020044B054A4A
:1015C8009B68C3F34233D35C034A1068D840704722
:1015D80000380240403C00081C0100200368DA681B
:1015E80022F49072DA605A6922F001025A612023CB
:1015F80080F83A30704700002DE9F0470668C26865
:101608003369C16923F44053134333610446836843
:101618000069F2680343606922F41642034322F02A
:101628000C020B431343F3607369A26923F44073FC
:101638001343B1F5004F73617A4B7CD19E4203D0BE
:1016480003F580639E4244D1FFF7B8FF192505FBD7
:1016580000F360684FF064094000B3FBF0F3B3FB9C
:10166800F9F34FEA0318FFF7A9FF636868435B00C3
:10167800B0FBF3F7FFF7A2FF636868435B00B0FBBA
:10168800F3F3B3FBF9F309FB1373DB003233B3FB5A
:10169800F9F35B0003F4F877FFF790FF626868439B
:1016A8005200B0FBF2FAFFF789FF636868435B00FA
:1016B800B0FBF3F3B3FBF9F309FB13A3DB003233FD
:1016C800B3FBF9F303F0070343443B44B360BDE8BD
:1016D800F087FFF763FF192505FB00F360684FF0FB
:1016E80064094000B3FBF0F3B3FBF9F34FEA0318C6
:1016F800FFF754FF636868435B00B0FBF3F7FFF73D
:101708004DFF636868435B00B0FBF3F3B3FBF9F389
:1017180009FB1373DB003233B3FBF9F35B0003F40B
:10172800F877FFF73BFF626868435200B0FBF2FAB4
:10173800FFF734FFB9E79E4202D03B4B9E4240D1AF
:10174800FFF73CFF676819254FF0640905FB00F3B4
:10175800BF00B3FBF7F3B3FBF9F31F01FFF72EFF4D
:10176800636868439B00B0FBF3F8FFF727FF6368E3
:1017780068439B00B0FBF3F3B3FBF9F309FB138356
:101788001B013233B3FBF9F303F0F008FFF716FF40
:10179800626868439200B0FBF2FAFFF70FFF6368D4
:1017A80068439B00B0FBF3F3B3FBF9F309FB13A306
:1017B8001B013233B3FBF9F303F00F0343EA0803C9
:1017C80083E7FFF7EBFE676819254FF0640905FB0F
:1017D80000F3BF00B3FBF7F3B3FBF9F31F01FFF707
:1017E800DDFE636868439B00B0FBF3F8FFF7D6FEA5
:1017F800636868439B00B0FBF3F3B3FBF9F309FBA1
:1018080013831B013233B3FBF9F303F0F008FFF73E
:10181800C5FE626868439200B0FBF2FAFFF7BEFEAD
:10182800BDE700BF0010014000140140F8B50446B0
:101838000E4617461D4621680B6836EA030301D198
:101848000020F8BD6B1CF7D095B92368DA6822F43C
:10185800D072DA605A6922F001025A61202384F8B2
:10186800393084F83A30002384F838300320F8BD42
:10187800FEF778FEC01B8542DDD2E6E710B50446C8
:1018880040B390F8393003F0FF021BB980F83820D4
:1018980001F0B2FD2268242384F83930D36823F498
:1018A8000053D3602046FFF7A7FE23681A6922F485
:1018B80090421A615A6922F02A025A61DA6842F49F
:1018C8000052DA6000202023E06384F8393084F87D
:1018D8003A3010BD012010BD2DE9F0411F4690F8A7
:1018E8003930202B04460D4690464FD100294AD066
:1018F800002A48D090F83830012B47D0012380F8CF
:1019080038300023C363212380F83930FEF72AFEDC
:10191800A4F824800646A4F82680E38C9BB26BB911
:101928003B46324640212046FFF780FFB0B92023CE
:1019380084F8393084F83800BDE8F081E38C013B45
:101948009BB2E384A368B3F5805F32463B464FF011
:10195800800120460ED1FFF769FF10B10320BDE8D2
:10196800F0812B882268C3F308035360236943B9C5
:101978000235D2E7FFF75AFF0028EFD123682A780B
:101988005A600135C9E70120BDE8F0810220BDE8B1
:10199800F08190F83A30202B1CD1C9B1C2B190F82F
:1019A8003830012B16D0C285828500232222C363DA
:1019B80080F83A2002688162516980F8383041F035
:1019C80001015161D16841F49071D16018467047A6
:1019D8000120704702207047704790F83A30222B58
:1019E80010B532D1836801690268B3F5805F836AF4
:1019F8001FD15268C9B9C2F3080223F8022B8362C7
:101A0800C48D013CA4B2C4856CB90368DA6822F4B9
:101A18009072DA605A6922F001025A61202380F834
:101A28003A3001F013FB002010BDD2B223F8012B8D
:101A3800E5E721B9591C526881621A70E0E75268DB
:101A4800591C816202F07F02F7E7022010BD70473F
:101A580003681A68D96870B5160704465D6907D126
:101A680096065AD58D0658D5BDE87040FFF7B5BF24
:101A780015F0010502D111F4907F4ED0D30705D59A
:101A8800CE0542BFE36B43F00103E363500704D57F
:101A98001DB1E36B43F00203E363930704D51DB163
:101AA800E36B43F00403E363160704D51DB1E36B4E
:101AB80043F00803E363E36B002B66D0950604D577
:101AC800880602D52046FFF788FF23685D69E26B28
:101AD8001107204602D415F040051AD0FFF77EFD05
:101AE80023685A69520610D55A69606B22F0400281
:101AF8005A6150B1254B0365FEF7B6FD002844D066
:101B0800606BBDE87040036D18472046FFF79FFFE4
:101B180070BDFFF79CFFE56370BD160627D50D065F
:101B280025D594F83920212A2FD1A268B2F5805FF3
:101B3800226A17D11188C1F308015960216979B95E
:101B480002322262E28C013A92B2E284EAB9DA689D
:101B580022F08002DA60DA6842F04002DA6070BD92
:101B68000132EEE7511C216212785A60EAE750060A
:101B78000BD54A0609D5DA6822F04002DA6020233C
:101B880084F839302046FFF727FF70BD991B0008FD
:101B980008B5806B0023C385C384FFF758FF08BDD1
:101BA80084B038B505AD85E80E000A9B012B0446C4
:101BB80026D1836B23F480338363C36823F48403BF
:101BC80023F04003C360C36823F44013C360119B30
:101BD800012B02BFC36843F48013C36000F0DEFB2F
:101BE800089B012B07D1A36843F00603A360A368F1
:101BF80043F02003A360BDE83840002004B07047DC
:101C0800C36843F04003C36000F0C8FB4FF480335F
:101C1800A363E5E7836843F001038360002070470E
:101C2800836823F0010383600020704708B5C36808
:101C3800012923F0C043C36008D1C36843F00053AF
:101C4800C3603220FEF794FC002008BD0029F8D1BB
:101C5800C36843F08043C360F3E7000084B02DE914
:101C6800F041044607A880E80E00119E0A9FA36B66
:101C78008846A6B943F40013A3630023C4F8003EC2
:101C8800D4F80038C4F800380C9B012B04F5006523
:101C98005ED1099939B9204600F09EF807E043F46F
:101CA8000023A363E9E71946204600F095F81021C0
:101CB800204600F06FF8204600F07EF800234FF031
:101CC800FF322B6119466B614FF09040AA614FF0CB
:101CD800FF0EEB6104F5106243453BD1002104F58A
:101CE800306208464FF0904E4FF0FF0C8B423ED1C9
:101CF8002B69012F23F480732B6108D1234B2B63AD
:101D08002B6B43F4803343F003032B632B6B0023CB
:101D1800A3616FF0804363611FB9A36943F01003A7
:101D2800A361A2691A4B1343A3610D9B1BB1A3695D
:101D380043F00803A361012E01BFA36943F0804368
:101D480043F00403A361BDE8F041002004B07047EC
:101D58000321A0E7D2F800C0BCF1000FB4BF1060A7
:101D6800116001331161C2F808E02032B4E7D2F8FB
:101D78000080B8F1000FB4BFC2F800E01060013174
:101D88001061C2F808C02032B0E700BF000180002F
:101D980000383C80890141F02001064A0161013A7E
:101DA80005D0036913F02003F9D1184670470320C2
:101DB800704700BF410D03001023064A0361013A32
:101DC80005D0036913F01003F9D1184670470320B2
:101DD800704700BF410D0300D0F800381943C0F820
:101DE80000180020704700F50062D0F8080810F0CD
:101DF800060012D0936803F00603022B0CD09368F8
:101E080003F00603062B07D0936803F00603042BA0
:101E180014BF0020022070470320704730B54B786C
:101E28000C78D0F81C5800F50062012B1BD1A34098
:101E38009BB22B4300F51060D36100EB44131A6882
:101E480012040ED48A68C8781D68C2F30A0242F0E8
:101E5800805242F4004242EA804040EA84502843DB
:101E68001860002030BD4FF48033A34000F5306087
:101E78002B4300EB4410D36103681B04F1D48B6837
:101E8800C9780268C3F30A0343F0805343F400435C
:101E980043EA814313430360E3E700F001B800001D
:101EA80070B54B78012B0E46054609784FF0200394
:101EB80026D100F5106213FB01231A6822F40042B0
:101EC8001A604FF000621A604FF080421A601F4A91
:101ED800013A01D1032070BD9C6814F08044F7D109
:101EE80010212846FFF756FF3178D5F81C28012322
:101EF8008B409BB222EA0303C5F81C38204670BD0C
:101F080000F5306213FB01231A6822F400421A60BC
:101F18004FF000621A604FF080421A600B4A013A93
:101F2800D8D0986810F01000F9D1D5F8043843F4E7
:101F38008063C5F80438D5F81C384FF480328A40DD
:101F480023EA0203C5F81C3870BD00BF410D030029
:101F5800F7B54B780C78012B4B6977D1202600F523
:101F6800106516FB04542669002B38D126F0FF565D
:101F780026F4C0162661266946F4002626612669DD
:101F8800F60CF6042661012A50D10C780E6905EB8F
:101F980044146661CE78012E0FD1D0F808480F7826
:101FA80014F4807F4FF0200414FB075427680CBFFB
:101FB80047F0005747F0805727600F7805EB471523
:101FC800012E2C6844F004442C6005D100929BB289
:101FD8003A46C96800F0EFF8002003B0F0BDF60CEF
:101FE800F604266126698F6826F0FF5626F4C01687
:101FF8002661DE19013EB6FBF7F7374ED4F810E03C
:1020080006EAC74646EA0E0626612769C3F31206A2
:102018003E432661CE78012E5AD1266926F0C04665
:102028002661266946F000562661ACE7CE78012E77
:10203800B3D0002BAED091F800E0D0F8347801246A
:1020480004FA0EF43C43C0F83448A3E700F53065C1
:1020580005EB44142569ED0CED042561256925F08F
:10206800FF5525F4C01525618D68FBB92369C5F3B3
:1020780012051D432561236943F400232361012AC6
:1020880004BFCB686361CB78012B0AD1D0F808383C
:1020980013F4807F23680CBF43F0005343F0805350
:1020A8002360236843F00443236095E70A4E2769B9
:1020B8002B44013BB3FBF5F306EAC3463E432661D6
:1020C8009BB226695D43C5F3120535432561D6E702
:1020D800012AAED159E700BF0000F81F4B78012B49
:1020E80070B50B784D6943D1202400F5106614FBB8
:1020F80003631C69CDB924F0FF5424F4C0141C6197
:102108001C6944F400241C611C69E40CE4041C618F
:102118000D7806EB4513012A1C6844F004441C6042
:102128001BD10A695A61002070BDE40CE4041C61EB
:102138001C6924F0FF5424F4C0141C618C68A54267
:1021480088BF4C611C6944F400241C614C691D69FA
:10215800C4F312042C431C61DAE74B69002BE2D06C
:10216800D0F834280123AB401343C0F83438DAE7F9
:1021780000F5306000EB43100369DB0CDB040361FE
:10218800036923F0FF5323F4C01303618B6805B17F
:102198004B61046944F4002404610469C3F3120325
:1021A8002343012A036104BFCB684361036843F0FA
:1021B80004430360B7E710B59DF808404CB90333F2
:1021C80000F5805023F0030300EB02320B449942E0
:1021D80001D1002010BD51F8040B1060F7E703325D
:1021E80022F003020A4400F58050914201D10846CA
:1021F8007047036841F8043BF7E74B780A78012BEE
:102208004FF020030BD100F5106013FB02000368A8
:10221800002B0BDB036823F08043036006E000F526
:10222800306013FB02000368002BF3DA036843F401
:1022380000130360002070474B780A78012B0CBF0D
:1022480000F5106000F53060202313FB02000368DE
:1022580023F400130360CB78023B012B9EBF036875
:1022680043F08053036000207047D0F8003823F40F
:10227800FE63C0F80038D0F80038090101F4FE61A7
:102288001943C0F800180020704708B5D0F8043882
:1022980023F00203C0F804380320FEF769F9002090
:1022A80008BD08B5D0F8043843F00203C0F8043874
:1022B8000320FEF75DF9002008BD426980691040DF
:1022C8007047D0F8183800F50060C0691840000C55
:1022D8007047D0F8183800F50060C069184080B21F
:1022E800704700F5306303EB411100F500608A6820
:1022F80040691040704710B5D0F81048D0F834380D
:1023080000EB4110CB4000F51060DB018068DBB2C8
:102318002343184010BD406900F001007047D0F811
:10232800003923F4FF6323F00703C0F8003900F5F0
:1023380000639A6802F00602042A02BFD0F8002956
:1023480042F00302C0F800295A6842F480725A60C9
:102358000020704710B50024C0F8104BD0F8104B7F
:1023680044F40024C0F8104BD0F8104B44F0180483
:10237800C0F8104BD0F8104B012900F5306344F039
:10238800C04408BF4FF08023C0F8104B04BFC0F80A
:10239800142BC0F8003B002010BD00000A4B013B85
:1023A80001D1032070470269002AF8DA0369064A56
:1023B80043F001030361013AF3D0036913F0010309
:1023C800F9D11846704700BF410D0300D0F8183204
:1023D8001BB10020C3F81402704702207047D0F8E0
:1023E8001C3210B5D0F818425BB194F80002FF28EF
:1023F80007D09B6894F8012221469847FF2384F868
:102408000032002010BD00004323038000487047BD
:1024180040000020432303800048704784000020C8
:102428004323038000487047D40000200A23038018
:1024380000487047C800002038B50546D0F8184253
:1024480001F046FAD5F81832C4F80C024BB1D5F8A9
:102458001C32D4F80402DB6804F5037198470020A5
:1024680038BD022038BD0000F8B50F7817F06003BA
:1024780006460C4623D0202B19D1CA884B78C2B106
:102488003906D0F818520BD5D0F81C1218468F68A8
:102498002946B847E2882946304600F09AFB06E00C
:1024A80085F8003285F80122294600F0A7FB0020B4
:1024B800F8BDD0F81C0284681846A047F7E74B78A7
:1024C8000A2BF4D101220149E7E700BFE40100200B
:1024D80010B58121044601F093F90121204601F04D
:1024E8008FF98221204601F08BF9D4F8183253B1C4
:1024F800D4F81C325B689847D4F8180201F096FAB1
:102508000023C4F81832002010BDF8B5037C044637
:102518007BBB4FF400730222812101F061F94FF473
:10252800007302220121204601F05AF908230322F0
:102538008221204601F054F94FF4077001F06EFA39
:102548000646C4F8180220B3D4F81C321B68984712
:10255800277C0025C6F81452C6F8185287B94FF4DC
:102568000073D6F804220121204601F0A3F9384669
:10257800F8BD40230222812101F032F94023D0E73F
:102588004023D6F804220121204601F093F9284679
:10259800F8BD0120F8BD19B1C0F81C120020704721
:1025A80002207047D0F818320020C3F80812C3F888
:1025B80010227047D0F818320020C3F80412704770
:1025C800D0F8182210B572B1D2F81442012364B9B8
:1025D800C2F814328121B2F81032D2F8082201F080
:1025E8005BF9204610BD022010BD184610BDD0F87A
:1025F800182210B562B1047C44B94FF40073D2F8C4
:102608000422012101F056F9002010BD4023F6E70D
:10261800022010BD08B580B1D0F8143213B10023E0
:10262800C0F8143209B1C0F81012012380F8FC3147
:10263800027001F097F8002008BD022008BD19B10A
:10264800C0F81412002070470220704708B501F046
:10265800B9F8002008BD08B5D0F814320BB902202B
:1026680008BD1B6898470028F9D108BD08B5D0F8FF
:1026780014325B689847002008BD38B5044600F559
:102688000275284600F075FA012394F80812C4F878
:10269800F431B4F80E32C4F8F83101F01F03012BFD
:1026A8000ED007D3022B10D001F08001204601F094
:1026B800B5F803E02946204600F0E6F8002038BDCA
:1026C8002946204600F0DAF9F8E72946204600F0C6
:1026D800EDF9F3E738B50446154611BBD0F8F431E7
:1026E800032B0FD1D0F80C31D0F8102193420BD91D
:1026F8009B1A9A4228BF1A46C0F80C3192B2294652
:1027080000F08BFA002038BDD0F814321B6923B1D1
:1027180090F8FC21032A00D19847204600F085FA5A
:10272800F0E7D0F814329B69002BEBD090F8FC212D
:10273800032AE7D19847E5E770B5134604460E46E5
:1027480000293DD1D0F8F421022A0FD1C569026AC7
:10275800954214D9AA1AC261194692B200F046FAF3
:1027680033461A461946204601F0A4F894F8003278
:10277800012B02D1002384F80032002070BD836948
:10278800B3FBF2F502FB153565B99A420AD8D0F8C1
:10279800F821934206D22A4600F028FAC4F8F851E4
:1027A8002B46DEE7D4F81432DB682BB194F8FC2111
:1027B800032A01D120469847204600F041FAD5E780
:1027C800D0F814325B69002BD7D090F8FC21032A8B
:1027D800D3D19847D1E738B50022044611464025A1
:1027E800402300F0FDFF2B46C4F810510022802141
:1027F800204600F0F5FF012384F8FC31D4F81832A4
:1028080025622BB1D4F8143221795B6820469847A9
:10281800002038BD01740020704790F8FC3180F822
:10282800FD31042380F8FC310020704790F8FD3119
:1028380080F8FC310020704708B590F8FC21032A85
:1028480004D1D0F81432DB6903B19847002008BDE1
:1028580000207047002070470020704708B501220B
:1028680080F8FC21D0F814220179526890470020A2
:1028780008BD10B58021044600F0D0FF2046002195
:10288800BDE8104000F0CABF37B54B7804460D4686
:10289800092B79D8DFE813F0C900E5007800D900E2
:1028A80078006D000A007800B9008D004B881A0A7C
:1028B800013A062A68D8DFE802F0041C296767494C
:1028C8005200D0F810321B68207C0DF106019847A1
:1028D800BDF80620002A67D0EB88002B64D09A4206
:1028E80028BF1A46ADF806200146204600F071F9C7
:1028F8005AE0027CD0F8143232B99B6A0DF1060016
:10290800984702234370E3E7DB6AF7E7DBB2052B5E
:102918003AD8DFE803F003070B0F1317D0F810328B
:102928005B68D1E7D0F810329B68CDE7D0F8103259
:10293800DB68C9E7D0F810321B69C5E7D0F8103258
:102948005B69C1E7D0F810329B69BDE7037CDBB94E
:10295800D0F814320DF106005B6B9847B8E7037C9A
:1029680093B9D0F814320DF106001B6B9847072372
:10297800C8E78B8843B9CB8833B990F8FC318D7898
:10298800032B05F07F0503D12046FFF772FF0BE00C
:1029980080F8FE51294600F071FF204600F045F905
:1029A8002DB1022384F8FC31002003B030BD01238F
:1029B800F8E78978304D01292970E5D890F8FC317D
:1029C800022B0CD0032BDFD1B1B9022380F8FC31E4
:1029D8004160FFF74BFE204600F027F9E4E70029A5
:1029E800F9D001210323416080F8FC312046FFF72C
:1029F80032FE0228EFD1C7E741680129EBD0C9B2FE
:102A0800FFF734FE29786160F0E7CA88012ABBD154
:102A180090F8FC31022B03D0032BB5D1011D64E7DC
:102A28000146002341F8083F5FE790F8FC31023B7C
:102A3800012BA9D80123C360D0F804320BB10323BA
:102A4800C360022204F10C014FE74B88012BABD184
:102A5800C4F80432D4F8143229469B6820469847B3
:102A6800B9E790F8FC31023B012B8DD84B88012B3C
:102A78009AD10023ECE700BFE501002038B590F8B3
:102A8800FC31032B04460D460DD10B79012B0AD8D6
:102A9800D0F814329B689847EB8813B9204600F0A9
:102AA800C4F8002038BDFFF7E4FEFAE770B50A78ED
:102AB8008E8802F06002202A04460D46F3B205D142
:102AC800D0F814329B689847002070BD4A78012AD4
:102AD8001CD02AD3032AF7D190F8FC21022A40D02F
:102AE800032A02D0FFF7C5FEEEE74A8822B95E0640
:102AF80002D0194600F092FED4F8143229469B6899
:102B080020469847204600F090F8DDE790F8FC2131
:102B1800022A26D0032AE5D14A88002AD4D15906A8
:102B2800F0D0194600F088FEE6E790F8FC21022A6A
:102B380017D0032AD6D103F07F0516F0800F00EBDB
:102B48000515194614BF143505F5827500F082FE87
:102B580068B101232B6002222946204600F039F88B
:102B6800B2E75A06B0D0194600F058FEACE7286024
:102B7800F1E70B7803704B784370CA788B7803EBD6
:102B8800022343804A790B7903EB02238380CA79B5
:102B98008B7903EB0223C380704730B588B10546B3
:102BA8002B1A15F8014BDBB2002CF9D15B0002336C
:102BB80013800B7003234B700138022310F8015F58
:102BC80005B930BD5A1CD2B2CD540233DBB28C5495
:102BD800F4E710B513460222C0F8F42183610A46CF
:102BE800C361002100F058FE002010BD08B513464F
:102BF8000A46002100F050FE002008BD10B513461B
:102C08000322C0F8F421C0F808310A46C0F80C3194
:102C1800002100F04FFE002010BD08B513460A46FB
:102C2800002100F047FE002008BD08B50423C0F8C5
:102C3800F43100231A46194600F02EFE002008BD84
:102C480008B50523C0F8F43100231A46194600F0E8
:102C580031FE002008BD00000C4B00025861586985
:102C680001435961A3F580634FF6FE70596941F03D
:102C78000201596102B9704759690140596159699E
:102C880041F001015961013AF4E700BF0004024034
:102C9800094B000258615A6911435961A3F58063D1
:102CA8005A6922F001021204120C5A615A6942F060
:102CB80001025A61704700BF00040240054A536987
:102CC80023F002031B041B0C014653610020FFF78D
:102CD800DFBF00BF00000240034A536943F002030C
:102CE8005361FFF7D5BF00BF0000024010B5884C04
:102CF8001F2363610520FDF73BFC636923F008038C
:102D08001B041B0C63610F20FDF732FC636943F061
:102D1800080363610F20FDF72BFC636923F00403AC
:102D28001B041B0C6361E920FFF7C8FF202100206A
:102D3800FFF7D2FF1120FFF7C1FF6420FDF718FC51
:102D4800D120FFF7BBFF00210846FFF7C5FF71211F
:102D58000020FFF7C1FF19210020FFF7BDFFD02099
:102D6800FFF7ACFF07210020FFF7B6FF0121002085
:102D7800FFF7B2FF08210020FFF7AEFF3620FFF76C
:102D88009DFF48210020FFF7A7FF3A20FFF796FF95
:102D980005210020FFF7A0FFC120FFF78FFF1021BA
:102DA8000020FFF799FF10210020FFF795FF02216F
:102DB8000020FFF791FF02210020FFF78DFFC020C0
:102DC800FFF77CFF00210846FFF786FF352100202A
:102DD800FFF782FF00210846FFF77EFF0021084623
:102DE800FFF77AFF01210020FFF776FF022100207C
:102DF800FFF772FFC520FFF761FF04210020FFF7EE
:102E08006BFFD220FFF75AFF01210020FFF764FF74
:102E180044210020FFF760FFC820FFF74FFF04217F
:102E28000020FFF759FF67210020FFF755FF3521E4
:102E38000020FFF751FF04210020FFF74DFF082174
:102E48000020FFF749FF06210020FFF745FF242156
:102E58000020FFF741FF01210020FFF73DFF372148
:102E68000020FFF739FF40210020FFF735FF03213D
:102E78000020FFF731FF10210020FFF72DFF082168
:102E88000020FFF729FF80210020FFF725FF002100
:102E98000846FFF721FF2A20FFF710FF0021084608
:102EA800FFF71AFF00210846FFF716FF0021084622
:102EB800FFF712FFEF210020FFF70EFF2B20FFF78F
:102EC800FDFE00210846FFF707FF00210846FFF72F
:102ED80003FF01210020FFF7FFFE8F210020FFF7ED
:102EE800FBFE2920FFF7EAFE2C20FFF7E7FE6369C7
:102EF800084A43F004036361FF231380064A1380E2
:102F0800064BF8221A80064B00221A8010BD00BF1B
:102F180000000240FC010020FE01002020020020E9
:102F280014020020F8B51D461C4B1B6804460F46CA
:102F380016463BB91A4B1B881C1A9B1A2E469FB281
:102F4800A5B20C462A20FFF7B9FE210A0020FFF798
:102F5800C3FE21460020FFF7BFFE310A0020FFF71D
:102F6800BBFE31460020FFF7B7FE2B20FFF7A6FE79
:102F7800390A0020FFF7B0FE39460020FFF7ACFE03
:102F8800290A0020FFF7A8FE29460020FFF7A4FE23
:102F98002C20BDE8F840FFF791BE00BF1C020020BE
:102FA8001A010020064B074A1968074829B11388F7
:102FB800028800210846FFF7B5BF03881288F9E7A1
:102FC8001C0200201A0100201801002010B50C4C2A
:102FD800636923F004031B041B0C6361FFF7E2FF22
:102FE800084A094B12881B880021013203FB022280
:102FF8000846FFF731FE636943F00403636110BDBF
:10300800000002401A0100201801002038B50C4CBD
:10301800636923F004031B041B0C63610546FFF777
:10302800C1FF084B084A1B881288E9B25A43280A8C
:10303800FFF712FE636943F00403636138BD00BF04
:10304800000002401A01002018010020354B83427D
:1030580010B565D1344C2378762B07D1334B012238
:103068001A7042214FF6FF73FEF736FC2378732B54
:1030780009D12E4B2B4800221A7042214FF6FF73BC
:103088000122FEF729FC2378642B09D1284B254817
:1030980000221A7042214FF6FF730122FEF71CFC32
:1030A8002378752B08D1224B1E4801221A70422121
:1030B8004FF6FF73FEF710FC2378562B08D11D4BF3
:1030C800184801221A7042214FF6FF73FEF704FCDC
:1030D8002378532B09D1174B124800221A7042212A
:1030E8004FF6FF730122FEF7F7FB23784C2B09D12B
:1030F800114B0C4800221A7042214FF6FF7301222F
:10310800FEF7EAFB2378522B0AD10B4B0548012224
:103118001A7042214FF6FF73BDE81040FEF7DCBB82
:1031280010BD00BF4C02002004020020E80100206E
:10313800E6010020E9010020E701002030B595B044
:103148003022002108A800F079FC0021142203A8ED
:1031580000F074FC00241D4B01941A6C42F080525C
:103168001A641B6C03F080530193019B184B029463
:103178001A6842F480421A601B6803F48043029381
:10318800029B012308934FF4803309934FF4800383
:103198000F9304231093A8230225119308A807234B
:1031A80013930E951295FDF7A9FF0F230393A02300
:1031B80005934FF4A053069321464FF4805303A878
:1031C80004950793FEF74AF915B030BD0038024060
:1031D800007000407FB51422002101A800F02EFCE9
:1031E8000F23019301A9012303480293FDF74EFA27
:1031F80007B05DF804FB00BF000802402DE9F0416C
:103208008AB0FDF789F9FFF799FF142200210DEB29
:10321800020000F013FC00245D4B01941A6B5D481A
:103228005D4D5E4F42F080021A631A6B02F0800215
:103238000192019A02941A6B42F001021A631A6B06
:1032480002F001020292029A03941A6B42F00202FF
:103258001A631A6B02F002020392039A04941A6B1F
:1032680042F004021A631B6B03F004032246049322
:103278000F21049BFDF7EAFA22464FF6FF714848F2
:10328800FDF7E4FA01260F2305A94248059306969F
:1032980007940894FDF7FAF905A94FF6FF7340481B
:1032A8000593069607940894FDF7F0F9FFF792FF47
:1032B80000F01EF93B4AAC604FF4165385E80C0049
:1032C80028460C236B61EC602C61AC61EC61FEF765
:1032D800D5FAFFF70BFD344B04F180441E6004F56A
:1032E8000234FFF773FE4FF47840FFF78FFE4FF478
:1032F8007A70FDF73DF963692C493343636163696B
:1033080043F00403324628466361FEF742FB284D2A
:10331800284E95F80080B8F1010F0FD1636923F0AA
:10332800010363614046FDF723F9636943F0010334
:1033380063614046FDF71CF900232B703B78012B95
:1033480063690CBF43F0020323F00203636196F83C
:103358000080B8F1010F0FD1636923F004036361A2
:103368004046FDF705F9636943F00403636140468D
:10337800FDF7FEF8002333700F4B1B78012B6369B0
:103388000CBF43F0080323F008036361C1E700BFE3
:1033980000380240000002404C020020E6010020F4
:1033A80000040240004C00401C02002004020020DF
:1033B800E8010020E9010020E70100207047000033
:1033C80082B00C4B002100915A6C42F480425A643E
:1033D8005A6C02F480420092009A01911A6C42F0F1
:1033E80080521A641B6C03F080530193019B02B056
:1033F800704700BF0038024010B5044688B0142258
:10340800002103A800F01AFB2268194B9A422DD11B
:1034180003F5F633002401941A6C164842F400228E
:103428001A641A6C02F400220192019A02941A6B2F
:1034380042F004021A631B6B03F004030293029B1D
:103448004FF440630393022304930123059303235A
:10345800069303A908230793FDF718F93420224699
:103468002146FDF7ABF83420FDF7DCF808B010BDB5
:10347800004C0040000802407047FEE7FEE7FEE708
:10348800FEE7704770477047FDF760B80148FEF7E0
:10349800DFBA00BF4C0200200148FDF75DBA00BF4B
:1034A800983A00200F49D1F8883043F47003C1F8E6
:1034B80088300D4B1A68002042F001021A609860AB
:1034C8001A6822F0847222F480321A60074A5A601D
:1034D8001A6822F480221A60D8604FF000638B606B
:1034E800704700BF00ED00E00038024010300024B3
:1034F80010B5094C094900222046FFF78BF8084906
:103508002046FFF79CF820460649FFF744F8204676
:10351800BDE81040FFF79AB80C28002030010020C1
:10352800080000202001002000207047002070477C
:1035380010B5064C064900222046FFF733F8054926
:103548002046FFF737F8002010BD00BF0C280020E8
:1035580034320020302A002010B5094CD4F8183233
:10356800D3F814320A4643B901462046FFF71AF841
:103578002046BDE81040FFF723B8012010BD00BF6A
:103588000C28002010B52B4C0A680146204600F094
:1035980019FB2378762B05D1274B28480121197070
:1035A800FFF7DAFF2378732B06D1234B2348002239
:1035B80001211A70FFF7D0FF23786C2B06D1204B1E
:1035C8001E48002201211A70FFF7C6FF2378722BCC
:1035D80005D11B4B194801211970FFF7BDFF23784E
:1035E800562B05D1174B154801211970FFF7B4FF69
:1035F8002378532B06D1134B1048002201211A704F
:10360800FFF7AAFF23784C2B06D10F4B0B4800225B
:1036180001211A70FFF7A0FF2378522B05D10A4B1E
:10362800064801211970FFF797FF0848FEF7DFFFEA
:10363800002010BD343A0020E8010020483C000872
:10364800E6010020E9010020E70100200C28002005
:1036580010B50368B3F1A04F86B025D14FF4C0531D
:1036680001930223029303230024049301A90A234C
:103678000E4805930394FDF709F80D4B5A6B42F079
:1036880080025A6300945A6C42F480425A645B6C1C
:1036980003F480430093432022462146009BFCF715
:1036A8008DFF4320FCF7BEFF06B010BD00000240AE
:1036B8000038024000F56F71D0F8EC03FEF7DDBF6B
:1036C8001C2303FB0103D0F8EC03D3F80422FFF713
:1036D80001B81C2303FB0103D0F8EC035A6CFFF775
:1036E8002BB8D0F8EC03FFF7A7B810B5C1680446AB
:1036F800003118BF0121D0F8EC03FFF78BF8D4F89C
:10370800EC03BDE81040FFF766B8000010B50446AA
:10371800D0F8EC03FFF781F82268D2F8003E43F0B6
:103728000103C2F8003E236A23B1034A136943F038
:103738000603136110BD00BF00ED00E0D0F8EC03F4
:10374800FFF774B8D0F8EC03FFF784B8D0F8EC03AF
:10375800FFF77EB8D0F8EC03FFF77EB8D0F8EC039B
:10376800FFF77CB808B502783ABB154B0421C3F8BB
:10377800EC03C0F820324FF0A04083E80300022198
:103788001846D9601A615A619961DA611A625A62F7
:10379800DA621A63FDF75FF808B1FFF70FFE8021C0
:1037A8000748FDF7A6FC402200210548FDF780FCEC
:1037B800802201210248FDF77BFC002008BD00BFE4
:1037C800983A002008B5D0F82002FDF7B0F8032891
:1037D8009ABF024B185C022008BD00BF4A3C000893
:1037E80010B51C46D0F8200213462246FDF772FB9E
:1037F80003289ABF014B185C022010BD4A3C000800
:1038080008B5D0F82002FDF793FB03289ABF024BB6
:10381800185C022008BD00BF4A3C000808B5D0F873
:103828002002FDF7F4FB03289ABF024B185C022024
:1038380008BD00BF4A3C000808B5D0F82002FDF7D3
:1038480012FC03289ABF024B185C022008BD00BF77
:103858004A3C000811F0800FD0F820324FF01C02CB
:103868001BBF01F07F0102FB013102FB013191F81E
:103878003A0008BF91F8FA017047000008B5D0F87F
:103888002002FDF715FB03289ABF024B185C0220A3
:1038980008BD00BF4A3C000808B5D0F82002FDF773
:1038A80096FB03289ABF024B185C022008BD00BF94
:1038B8004A3C000808B5D0F82002FDF75CFB032855
:1038C8009ABF024B185C022008BD00BF4A3C0008A2
:1038D80008B5D0F82002FDF772FB08BD12230B8053
:1038E800004870474C01002004230B8000487047B3
:1038F8006001002010B5044C04480A462146FFF731
:103908004CF9204610BD00BF883E0020673C0008E7
:1039180010B5044C04480A462146FFF73EF92046F4
:1039280010BD00BF883E00207A3C000810B5044C4A
:1039380004480A462146FFF730F9204610BD00BF6B
:10394800883E0020903C000810B5044C04480A4604
:103958002146FFF722F9204610BD00BF883E00200F
:103968004E3C000810B5044C04480A462146FFF7AF
:1039780014F9204610BD00BF883E0020593C0008BD
:10398800DFF834D0002103E00C4B5B58435004317E
:103998000B480C4B42189A42F6D30B4A02E000231C
:1039A80042F8043B094B9A42F9D3FFF77BFD00F03C
:1039B80011F8FFF723FC704700000220B03C000814
:1039C80000000020C8010020C80100208C40002011
:1039D800FEE7000070B50D4E0D4CA41BA410002589
:1039E800A54209D10B4E0C4C00F012F9A41BA410EF
:1039F8000025A54205D170BD56F8253098470135F8
:103A0800EEE756F8253098470135F2E7A83C00085C
:103A1800A83C0008A83C0008AC3C0008024B014642
:103A2800186800F061B800BF64010020024B01462D
:103A3800186800F00BB800BF640100200244034678
:103A4800934200D1704703F8011BF9E738B50546E2
:103A5800002945D051F8043C0C1F002BB8BFE418CE
:103A680000F0C5F81F4A1368104633B96360146044
:103A78002846BDE8384000F0BBB8A3420CD92168FD
:103A88006218934204BF1A685B68636004BF5218E7
:103A980022600460ECE713465A680AB1A242FAD9D8
:103AA80019685818A0420BD120680144581882425E
:103AB8001960DDD1106852685A6001441960D7E76F
:103AC80002D90C232B60D3E7206821188A4204BF4F
:103AD80011685268626004BF091821605C60C7E71A
:103AE80038BD00BFEC01002070B5CD1C25F00305E2
:103AF80008350C2D38BF0C25002D064601DBA942E0
:103B080003D90C233360002070BD00F070F8234AFD
:103B18001468214691B9224C23681BB9304600F03D
:103B280041F820602946304600F03CF8431C26D175
:103B38000C233360304600F05BF8E4E70B685B1B4E
:103B48001AD40B2B0FD90B60CD50CC18304600F08F
:103B58004FF804F10B00231D20F00700C31A1BD0F7
:103B68005A42E25070BD8C420DBF63684B68636077
:103B7800136018BF0C46E9E70C464968CAE7C41C3D
:103B880024F00304A04205D0211A304600F00AF8B8
:103B98000130CDD02560D9E770BD00BFEC01002011
:103BA800F001002038B5064C00230546084623607E
:103BB80000F020F8431C02D1236803B12B6038BD04
:103BC8008840002070B5044602B970BD234611F83C
:103BD800015B03F8015B561E1DB91444A34203D1CF
:103BE80070BD1C463246EFE703F8015BF6E7704705
:103BF80070470000044B1968024609B90349196067
:103C0800186802441A607047F40100208C400020B4
:103C1800F8B500BFF8BC08BC9E467047F8B500BFB1
:083C2800F8BC08BC9E46704781
:103C3000000000000000000001020304060708095C
:103C4000000000000102030442000002010243449C
:103C50004320436F6E6669670043444320496E7496
:103C60006572666163650053544D6963726F656C7C
:103C7000656374726F6E6963730053544D33322001
:103C80005669727475616C20436F6D506F72740069
:103C900030303030303030303030314100000000D2
:083CA00058C5FF7F0100000080
:043CA800AD01000862
:043CAC008901000882
:103CB000010000001000000013250008D9240008AE
:103CC0007124000800000000E7230008D523000845
:103CD0004124000800000000000000000000000077
:103CE0001D24000811240008292400083524000898
:103CF00009024300020100C032090400000102026F
:103D00000100052400100105240100010424020221
:103D100005240600010705820308001009040100BC
:103D2000020A0000000705010240000007058102A9
:103D30004000000009024300020100C032090400F3
:103D40000001020201000524001001052401000108
:103D5000042402020524060001070582030800105E
:103D600009040100020A0000000705010200020028
:103D700007058102000200000A0600020000004060
:103D80000100000009074300020104C032090400D9
:103D900000010202010005240010010524010001B8
:103DA000042402020524060001070582030800FF1F
:103DB00009040100020A000000070501024000009A
:103DC0000705810240000000EF00A3010024F40079
:103DD0003935000831350008353500088D350008C3
:103DE000E5380008F1380008FD38000819390008E6
:103DF00035390008513900086D39000812010002F8
:103E00000202004083044057000201020301000047
:103E10000403090468010020000000000000000005
:103E20000000000000000000000000000000000092
:103E30000000000000000000000000000000000082
:103E40000000000000000000000000000000000072
:103E50000000000000000000000000000000000062
:103E60000000000000000000000000000000000052
:083E700000000000000000004A
:04000005080039892D
:00000001FF
